:020000020000FC
:020000007CC1C1
:0200080004C032
:10000E00C4C0E6C0DFB6CF93DF93FF93EF93FF2715
:10001E00C82DC0FF24C0E8E9C191D0812197D9F441
:10002E00C92DC0FD13C0C498C92DC1609C2EE0E936
:10003E00C191D081CC2331F4DD2321F4C82DCE7FA4
:10004E008C2E0DC0E8E9C193D08309C0C49AC82D87
:10005E00CE7F8C2E04C0EA95C193D08300C0C82DEC
:10006E00C1FF24C0EAE9C191D0812197D9F4C92DED
:10007E00C1FD13C0C598C92DC2609C2EE2E9C19185
:10008E00D081CC2331F4DD2321F4C82DCD7F8C2EED
:10009E000DC0EAE9C193D08309C0C59AC82DCD7FA2
:1000AE008C2E04C0EA95C193D08300C0C82DC2FF28
:1000BE0024C0ECE9C191D0812197D9F4C92DC2FD9C
:1000CE0013C0C698C92DC4609C2EE4E9C191D0819D
:1000DE00CC2331F4DD2321F4C82DCB7F8C2E0DC023
:1000EE00ECE9C193D08309C0C69AC82DCB7F8C2E64
:1000FE0004C0EA95C193D08300C0C82DC3FF24C0AD
:10010E00EEE9C191D0812197D9F4C92DC3FD13C059
:10011E00C798C92DC8609C2EE6E9C191D081CC2329
:10012E0031F4DD2321F4C82DC77F8C2E0DC0EEE9EE
:10013E00C193D08309C0C79AC82DC77F8C2E04C027
:10014E00EA95C193D08300C0C091A100D091A200C6
:10015E00CC2311F4DD2399F0C091A300D091A4001B
:10016E00219729F0C093A300D093A40008C0C09398
:10017E00A100C093A200C091A000CF60C8BBEF91B8
:10018E00FF91DF91CF91DFBE1895DFB60F93FF93EE
:10019E00EF93DF93CF930CB15C9913C0FF27E32D40
:1001AE0001930D3051F4E0E6DD27C4E70191099388
:1001BE000D30E1F7E0E6816003C0E43709F4E0E6D4
:1001CE003E2ECF91DF91EF91FF910F91DFBE1895EB
:1001DE00DFB60F93121421F455980F91DFBE1895C8
:1001EE00EF93FF93FF27E22D0191E83809F4E0E643
:1001FE002E2E0CB9FF91EF91F0CF10E200270A9549
:10020E00F1F71A95E1F70895F8941214FF27E12DEE
:10021E000193E83809F4E0E61E2E559A7894089575
:10022E005527442760E13695279510F4400F511F4E
:10023E0057954795379527956A95B9F70895C72E1F
:10024E00C72FDD270991003318F00A3308F4FACFCF
:10025E0021977C2F7C19D1F07630C0F47C2FEEEBF9
:10026E00F6E07724662411270A910053C89531963B
:10027E00202DC8953196302DD3DF620E731E30F0CF
:10028E00CC1591F7442311F4889408950894089599
:10029E00C8953196002039F0002DFF93EF93B4DF0F
:1002AE00EF91FF91F5CF0895FF270191EF93ACDF0A
:1002BE00EF91FF270D3009F0F8CF0AE0A5DF089582
:1002CE00C72FDD270881003211F4C395FBCF7C2F99
:1002DE000895C72FDD27C895002011F47C2F0895AF
:1002EE0031960991001509F4F6CF08950FED0DBF63
:1002FE0000E6102E202E00E6302E882700EF07BBDA
:10030E000FEF08BB56B208E90AB900E409B9FF2796
:10031E00F093A100F093A2009924882400270FBD2A
:10032E000DE00EBD00E00BBD0DE30ABD00E409BFFC
:10033E00E091A100F091A200E093A300F093A4003D
:10034E00789481FF0AC006B30F70051529F09A95AF
:10035E0021F4502EBCD001C09FEF80FFF2CFF89455
:10036E008E7F74E7ADDFE4E4F6E0B3DF11F441D045
:10037E00DFCFE6E4F6E0ADDF11F463D0D9CFE0E5F0
:10038E00F6E0A7DF11F46BD0D3CFECE5F6E0A1DFFA
:10039E0011F473D0CDCFE4E6F6E09BDF11F48CD0F0
:1003AE00C7CFEEE6F6E095DF11F4A4D0C1CFEAE7B1
:1003BE00F6E08FDF11F4E3D0BBCFE0E8F6E089DFA3
:1003CE0011F4F8D0B5CFE2E7F6E083DF11F4CDD02B
:1003DE00AFCFE8E8F6E07DDF11F4FCD0A9CFEEE870
:1003EE00F6E077DF11F429D0A3CFEAE9F6E050DF8B
:1003FE00A7CFE2EAF6E04CDF0895C72FDD2708818C
:10040E000D3011F418940895003338F0043328F4A5
:10041E000053739588949894089598940894089529
:10042E00102F01E08894112319F0001F1A95FCCFAC
:10043E000895EAE9F6E02CDF0895E4E9F6E028DF16
:10044E00089544243DDFD9DF29F098F30C5FE8DFEF
:10045E00402AF8CF409408B3042108BBEECF4424C1
:10046E002FDFCBDF29F028F30C5FDADF402AF8CF3D
:10047E0008B3042908BBE1CFDCCF08B3007F16B365
:10048E001F70102B78E0111F10F001E301C000E384
:10049E00BBDE7A95C1F700E2B7DEE091A100F091E4
:1004AE00A200EF2B11F001E301C000E3ADDE0DE081
:1004BE00ABDE0AE0A9DE089503DF9FDF0230E0F62F
:1004CE00889400FB81F906B30F70502EB6CF16B389
:1004DE0074E0110F7A95E9F774E0110F10F001E353
:1004EE0001C000E391DE7A95C1F70DE08DDE0AE0E2
:1004FE008BDE0895E5DE81DFB9F1B0F1402EE0DE4E
:10050E009EDE90F1662011F4772071F10FE0071551
:10051E0058F124D0A62CB72CD3DE91DE28F10FE0B3
:10052E00071510F11BD0042D000FF894FF27E8E8F3
:10053E00E00FA192B082E95F61927082E95FA192B1
:10054E00B082042D0C5F6CDF18B3102B18BB042D7A
:10055E0067DF802A0095902278946FCF04E0660CB6
:10056E00771C0A95E1F7089564CFAADE46DFE1F322
:10057E00D8F3F89455DF0095802278945ECFA0DEF4
:10058E003CDF91F388F3402E4BDF182D102361F3DF
:10059E00F894192D102311F078944BCF042D000FE1
:1005AE00FF27E8E8E00F61907080E15F6192708252
:1005BE00789443CF182D74E01295111F10F000E3BC
:1005CE0001C001E321DE7A95C1F70DE01DDE0AE0E0
:1005DE001BDE089575DE33DE38F2F894772049F489
:1005EE00662039F4FF27F093A100F093A2007894CF
:1005FE0024CFB4DFFF27E1EA61927082E3EA6192D1
:10060E0070825EDEEE2714E0F8DE68F0023058F4F9
:10061E0000950170EE0FE02B1A95B1F7E295E0937D
:10062E00A00078940ACFFF27F093A100F093A200C8
:04063E007894FFCEDF
:100644003F00616374697661746500006465616389
:100654007469766174650000737461747573000065
:100664006368616E67657300000061726D006469A0
:100674007361726D000072657365740074696D65F1
:100684007273000073616665000068656C6C6F00CE
:100694006F6B0D0A00006572726F720D0A00446F71
:1006A40075626C65466F7820492F4F205265762E0F
:1006B40020312E32610D0A00000001000A0064009E
:0406C400E803102710
:00000001FF
